 regwipe

 Timestamp is 4b00ff65 (Mon Nov 16 16:29:41 2009)

 Preferred load address is 00400000

 Start         Length     Name                   Class
 0001:00000000 00003076H .text                   CODE
 0001:00003080 000001d2H .text$x                 CODE
 0002:00000000 00000160H .idata$5                DATA
 0002:00000160 0000009cH .rdata                  DATA
 0002:00000200 00000238H .xdata$x                DATA
 0002:00000438 00000078H .idata$2                DATA
 0002:000004b0 00000014H .idata$3                DATA
 0002:000004c4 00000160H .idata$4                DATA
 0002:00000624 000003e8H .idata$6                DATA
 0002:00000a0c 00000000H .edata                  DATA
 0003:00000000 00000004H .CRT$XCA                DATA
 0003:00000004 00000014H .CRT$XCU                DATA
 0003:00000018 00000004H .CRT$XCZ                DATA
 0003:0000001c 00000004H .CRT$XIA                DATA
 0003:00000020 00000004H .CRT$XIZ                DATA
 0003:00000030 00000ae4H .data                   DATA
 0003:00000b18 00000074H .bss                    DATA
 0004:00000000 00000058H .rsrc$01                DATA
 0004:00000060 00000360H .rsrc$02                DATA

  Address         Publics by Value              Rva+Base     Lib:Object

 0001:00000000       ?setodscallback@@YAXP6AXPBD@Z@Z 00401000 f   debugx.obj
 0001:00000010       ?odsproc@@YAXPBD@Z         00401010 f   debugx.obj
 0001:00000030       ?GetTempPathA@@YAXAAVCString@@@Z 00401030 f   debugx.obj
 0001:000000b0       ?GetTempFileNameA@@YA?AVCString@@XZ 004010b0 f   debugx.obj
 0001:00000170       ?vin@@YAXPBD@Z             00401170 f   debugx.obj
 0001:00000240       ?vin@@YAXH@Z               00401240 f   debugx.obj
 0001:000002b0       ?vin@@YAXAAVCStringArray@@@Z 004012b0 f   debugx.obj
 0001:00000390       ?ods@@YAXPBDZZ             00401390 f   debugx.obj
 0001:00000400       ?odsnl@@YAXPBDZZ           00401400 f   debugx.obj
 0001:00000480       ?ode@@YAXPBDZZ             00401480 f   debugx.obj
 0001:00000540       ?log@@YAXFPBGZZ            00401540 f   debugx.obj
 0001:00000620       ?log@@YAXFPBDZZ            00401620 f   debugx.obj
 0001:000006a0       ?HexDump@@YAXKKK@Z         004016a0 f   debugx.obj
 0001:00000890       ?LocateNtdllEntryPoints@@YAEXZ 00401890 f   mem_nt.obj
 0001:000008d0       ?BBNtMapViewOfSection@@YAJPAX0PAPAXKKPAT_LARGE_INTEGER@@PAKW4_SECTION_INHERIT@@KK@Z 004018d0 f   mem_nt.obj
 0001:00000920       ?BBNtUnmapViewOfSection@@YAJPAX0@Z 00401920 f   mem_nt.obj
 0001:00000940       ?BBRtlInitUnicodeString@@YAXPAU_UNICODE_STRING@@PBG@Z 00401940 f   mem_nt.obj
 0001:00000960       ?BBNtOpenSection@@YAJPAPAXKPAU_OBJECT_ATTRIBUTES@@@Z 00401960 f   mem_nt.obj
 0001:00000980       ?BBMmGetPhysicalAddress@@YA?AT_LARGE_INTEGER@@PAX@Z 00401980 f   mem_nt.obj
 0001:000009a0       ?BBRtlNtStatusToDosError@@YAKJ@Z 004019a0 f   mem_nt.obj
 0001:000009c0       ?IsWinNTFamily@@YAHXZ      004019c0 f   mem_os.obj
 0001:000009d0       ?IsWin9xFamily@@YAHXZ      004019d0 f   mem_os.obj
 0001:000009f0       ?IsWin98@@YAHXZ            004019f0 f   mem_os.obj
 0001:00000a40       ?IsWin98SE@@YAHXZ          00401a40 f   mem_os.obj
 0001:00000a90       ?IsWinME@@YAHXZ            00401a90 f   mem_os.obj
 0001:00000ac0       ?IsPreWin2k@@YAHXZ         00401ac0 f   mem_os.obj
 0001:00000b10       ?IsWin2k@@YAHXZ            00401b10 f   mem_os.obj
 0001:00000b50       ?IsWinXP@@YAHPAG@Z         00401b50 f   mem_os.obj
 0001:00000ba0       ?IsWinVista@@YAHXZ         00401ba0 f   mem_os.obj
 0001:00000be0       ?IsWinNT@@YAHXZ            00401be0 f   mem_os.obj
 0001:00000c20       ?IsNTFS@@YAHPBD@Z          00401c20 f   mem_os.obj
 0001:00000c70       ?IsWin7@@YAHXZ             00401c70 f   mem_os.obj
 0001:00000cb0       ?error@@YAXJPAD@Z          00401cb0 f   mem_phys.obj
 0001:00000d00       ?OpenPhysicalMemory@@YAPAXXZ 00401d00 f   mem_phys.obj
 0001:00000d90       ?UnmapPhysicalMemory@@YAXK@Z 00401d90 f   mem_phys.obj
 0001:00000dc0       ?MapPhysicalMemory@@YAEPAXPAK11@Z 00401dc0 f   mem_phys.obj
 0001:00000e20       ?mread@@YAKPAX_J@Z         00401e20 f   mem_phys.obj
 0001:00000e60       ?mreadbuf@@YAHPAX_JPAEK@Z  00401e60 f   mem_phys.obj
 0001:00000ef0       ?TransV2P@@YAKPAXK@Z       00401ef0 f   mem_phys.obj
 0001:00000f60       ?read_unicode_string@@YAHPAX0PAG@Z 00401f60 f   mem_phys.obj
 0001:00000fe0       ?read_unicode_string_on_memory@@YAHPAX_JPAG@Z 00401fe0 f   mem_phys.obj
 0001:00001030       ?AddWithoutDuplicate@@YAXAAVCDWordArray@@K@Z 00402030 f   mem_reg.obj
 0001:00001060       ?HiveList@@YAXPAXAAVCDWordArray@@@Z 00402060 f   mem_reg.obj
 0001:00001130       ?printNTTime@@YAXPAU_FILETIME@@H@Z 00402130 f   mem_reg.obj
 0001:000011c0       ?printNK@@YAXPAU_CM_KEY_NODE@@H@Z 004021c0 f   mem_reg.obj
 0001:00001250       ?ParseCell@@YAHPAXQAU_DUAL@@KHKPAD@Z 00402250 f   mem_reg.obj
 0001:00001780       ?WalkOnCell@@YAHQAXQAU_DUAL@@KFKQAD@Z 00402780 f   mem_reg.obj
 0001:00001850       ?MakeTree@@YAXPAXAAVCDWordArray@@@Z 00402850 f   mem_reg.obj
 0001:00001a90       ?SearchBee@@YAXPAXPAEK_KAAVCDWordArray@@@Z 00402a90 f   mem_reg.obj
 0001:00001c00       ?HiveScan@@YAHPAXAAVCDWordArray@@@Z 00402c00 f   mem_reg.obj
 0001:00001d60       ?guess_dtb@@YAKPAX_K@Z     00402d60 f   mem_x86.obj
 0001:00001ed0       ?GetVersionText@@YA?AVCString@@PAUHINSTANCE__@@@Z 00402ed0 f   regwipe.obj
 0001:00001fa0       ?ShowUsage@@YAXXZ          00402fa0 f   regwipe.obj
 0001:00002010       ?DbgProc@@YAXPBD@Z         00403010 f   regwipe.obj
 0001:00002020       ?CtrlHandler@@YGHK@Z       00403020 f   regwipe.obj
 0001:00002030       ?Init@@YAHPAX@Z            00403030 f   regwipe.obj
 0001:000020f0       _main                      004030f0 f   regwipe.obj
 0001:000024c0       ?ShuffleArg@?$CSimpleOptTempl@D@@AAEXHH@Z 004034c0 f i regwipe.obj
 0001:00002510       ?LookupOption@?$CSimpleOptTempl@D@@ABEHPBD@Z 00403510 f i regwipe.obj
 0001:000025d0       ?LookupOption@?$CSimpleOptTempl@D@@ABEHD@Z 004035d0 f i regwipe.obj
 0001:00002610       ?FindEquals@?$CSimpleOptTempl@D@@ABEPADPAD@Z 00403610 f i regwipe.obj
 0001:00002640       _DllGetVersion@8           00403640 f   verinfo.obj
 0001:00002730       ??0CFileVersionInfo@@QAE@XZ 00403730 f   verinfo.obj
 0001:00002750       ??_GCFileVersionInfo@@UAEPAXI@Z 00403750 f i verinfo.obj
 0001:00002750       ??_ECFileVersionInfo@@UAEPAXI@Z 00403750 f i verinfo.obj
 0001:00002770       ??1CFileVersionInfo@@UAE@XZ 00403770 f   verinfo.obj
 0001:00002780       ?Open@CFileVersionInfo@@QAEHPAUHINSTANCE__@@@Z 00403780 f   verinfo.obj
 0001:000027e0       ?Open@CFileVersionInfo@@QAEHPBD@Z 004037e0 f   verinfo.obj
 0001:00002820       ?GetVersionInfo@CFileVersionInfo@@IAEHPBD@Z 00403820 f   verinfo.obj
 0001:000028c0       ?QueryVersionTrans@CFileVersionInfo@@IAEHXZ 004038c0 f   verinfo.obj
 0001:00002920       ?Close@CFileVersionInfo@@QAEXXZ 00403920 f   verinfo.obj
 0001:00002960       ?QueryStringValue@CFileVersionInfo@@QBEHPBDPADH@Z 00403960 f   verinfo.obj
 0001:00002a90       ?QueryStringValue@CFileVersionInfo@@QBEHHPADH@Z 00403a90 f   verinfo.obj
 0001:00002ac0       ?GetVerStringName@CFileVersionInfo@@QAEPBDH@Z 00403ac0 f   verinfo.obj
 0001:00002ae0       ?FindTrans@CFileVersionInfo@@QBEHGG@Z 00403ae0 f   verinfo.obj
 0001:00002b20       ?SetTrans@CFileVersionInfo@@QAEHGG@Z 00403b20 f   verinfo.obj
 0001:00002b90       ?GetTransByIndex@CFileVersionInfo@@QBEKI@Z 00403b90 f   verinfo.obj
 0001:00002bb0       ?SetTransIndex@CFileVersionInfo@@QAEHI@Z 00403bb0 f   verinfo.obj
 0001:00002bf0       ?GetLIDName@CFileVersionInfo@@SAHGPADH@Z 00403bf0 f   verinfo.obj
 0001:00002c20       ?GetCPName@CFileVersionInfo@@SAHGPAPBD@Z 00403c20 f   verinfo.obj
 0001:00002d00       _OutputDebugStringA@4      00403d00 f   kernel32:KERNEL32.dll
 0001:00002d06       _GetTempPathA@8            00403d06 f   kernel32:KERNEL32.dll
 0001:00002d0c       _GetTickCount@0            00403d0c f   kernel32:KERNEL32.dll
 0001:00002d12       _LocalFree@4               00403d12 f   kernel32:KERNEL32.dll
 0001:00002d18       _FormatMessageA@28         00403d18 f   kernel32:KERNEL32.dll
 0001:00002d1e       _GetSystemDefaultLangID@0  00403d1e f   kernel32:KERNEL32.dll
 0001:00002d24       _GetLastError@0            00403d24 f   kernel32:KERNEL32.dll
 0001:00002d2a       _WideCharToMultiByte@32    00403d2a f   kernel32:KERNEL32.dll
 0001:00002d30       _GetProcAddress@8          00403d30 f   kernel32:KERNEL32.dll
 0001:00002d36       _GetModuleHandleA@4        00403d36 f   kernel32:KERNEL32.dll
 0001:00002d3c       _FreeLibrary@4             00403d3c f   kernel32:KERNEL32.dll
 0001:00002d42       _LoadLibraryA@4            00403d42 f   kernel32:KERNEL32.dll
 0001:00002d48       _GetVersion@0              00403d48 f   kernel32:KERNEL32.dll
 0001:00002d4e       _GetVersionExA@4           00403d4e f   kernel32:KERNEL32.dll
 0001:00002d54       _lstrcmpiA@8               00403d54 f   kernel32:KERNEL32.dll
 0001:00002d5a       _GetVolumeInformationA@32  00403d5a f   kernel32:KERNEL32.dll
 0001:00002d60       _UnmapViewOfFile@4         00403d60 f   kernel32:KERNEL32.dll
 0001:00002d66       _MapViewOfFile@20          00403d66 f   kernel32:KERNEL32.dll
 0001:00002d6c       _IsBadReadPtr@8            00403d6c f   kernel32:KERNEL32.dll
 0001:00002d72       _IsBadWritePtr@8           00403d72 f   kernel32:KERNEL32.dll
 0001:00002d78       _FileTimeToSystemTime@8    00403d78 f   kernel32:KERNEL32.dll
 0001:00002d7e       _GlobalMemoryStatusEx@4    00403d7e f   kernel32:KERNEL32.dll
 0001:00002d84       _CloseHandle@4             00403d84 f   kernel32:KERNEL32.dll
 0001:00002d8a       _GetCommandLineA@0         00403d8a f   kernel32:KERNEL32.dll
 0001:00002d90       _GetModuleFileNameA@12     00403d90 f   kernel32:KERNEL32.dll
 0001:00002d96       _lstrcpynA@12              00403d96 f   kernel32:KERNEL32.dll
 0001:00002d9c       _VerLanguageNameA@12       00403d9c f   kernel32:KERNEL32.dll
 0001:00002da2       _wsprintfA                 00403da2 f   user32:USER32.dll
 0001:00002da8       _ShellExecuteA@24          00403da8 f   shell32:SHELL32.dll
 0001:00002dae       ?Delete@CString@@QAEHHH@Z  00403dae f   mfc42:MFC42.DLL
 0001:00002db4       ??1CString@@QAE@XZ         00403db4 f   mfc42:MFC42.DLL
 0001:00002dba       ?Right@CString@@QBE?AV1@H@Z 00403dba f   mfc42:MFC42.DLL
 0001:00002dc0       ?ReleaseBuffer@CString@@QAEXH@Z 00403dc0 f   mfc42:MFC42.DLL
 0001:00002dc6       ?GetBuffer@CString@@QAEPADH@Z 00403dc6 f   mfc42:MFC42.DLL
 0001:00002dcc       ??0CString@@QAE@ABV0@@Z    00403dcc f   mfc42:MFC42.DLL
 0001:00002dd2       ?Format@CString@@QAAXPBDZZ 00403dd2 f   mfc42:MFC42.DLL
 0001:00002dd8       ??0CString@@QAE@XZ         00403dd8 f   mfc42:MFC42.DLL
 0001:00002dde       ??1CStdioFile@@UAE@XZ      00403dde f   mfc42:MFC42.DLL
 0001:00002de4       ?Close@CStdioFile@@UAEXXZ  00403de4 f   mfc42:MFC42.DLL
 0001:00002dea       ?WriteString@CStdioFile@@UAEXPBD@Z 00403dea f   mfc42:MFC42.DLL
 0001:00002df0       ?Open@CStdioFile@@UAEHPBDIPAVCFileException@@@Z 00403df0 f   mfc42:MFC42.DLL
 0001:00002df6       ??0CStdioFile@@QAE@XZ      00403df6 f   mfc42:MFC42.DLL
 0001:00002dfc       ?FormatV@CString@@QAEXPBDPAD@Z 00403dfc f   mfc42:MFC42.DLL
 0001:00002e02       ?SetAtGrow@CDWordArray@@QAEXHK@Z 00403e02 f   mfc42:MFC42.DLL
 0001:00002e08       ?Replace@CString@@QAEHPBD0@Z 00403e08 f   mfc42:MFC42.DLL
 0001:00002e0e       ??0CString@@QAE@PBD@Z      00403e0e f   mfc42:MFC42.DLL
 0001:00002e14       ?SetSize@CDWordArray@@QAEXHH@Z 00403e14 f   mfc42:MFC42.DLL
 0001:00002e1a       ??1CDWordArray@@UAE@XZ     00403e1a f   mfc42:MFC42.DLL
 0001:00002e20       ??0CDWordArray@@QAE@XZ     00403e20 f   mfc42:MFC42.DLL
 0001:00002e26       ?AfxWinInit@@YGHPAUHINSTANCE__@@0PADH@Z 00403e26 f   mfc42:MFC42.DLL
 0001:00002e2c       ??3@YAXPAX@Z               00403e2c f   mfc42:MFC42.DLL
 0001:00002e32       __mbscmp                   00403e32 f   msvcrt:MSVCRT.dll
 0001:00002e38       ___CxxFrameHandler         00403e38 f   msvcrt:MSVCRT.dll
 0001:00002e40       _wcslen                    00403e40 f   msvcrt:MSVCRT.dll
 0001:00002e46       _isalnum                   00403e46 f   msvcrt:MSVCRT.dll
 0001:00002e4c       _printf                    00403e4c f   msvcrt:MSVCRT.dll
 0001:00002e52       _wcsncpy                   00403e52 f   msvcrt:MSVCRT.dll
 0001:00002e58       _free                      00403e58 f   msvcrt:MSVCRT.dll
 0001:00002e5e       _strncpy                   00403e5e f   msvcrt:MSVCRT.dll
 0001:00002e64       _malloc                    00403e64 f   msvcrt:MSVCRT.dll
 0001:00002e6a       _strncat                   00403e6a f   msvcrt:MSVCRT.dll
 0001:00002e70       __chkstk                   00403e70 f   msvcrt:chkstk.obj
 0001:00002e70       __alloca_probe             00403e70 f   msvcrt:chkstk.obj
 0001:00002ea0       _strncmp                   00403ea0 f   msvcrt:MSVCRT.dll
 0001:00002ea6       _atoi                      00403ea6 f   msvcrt:MSVCRT.dll
 0001:00002eac       _sscanf                    00403eac f   msvcrt:MSVCRT.dll
 0001:00002eb2       _mainCRTStartup            00403eb2 f   msvcrt:crtexe.obj
 0001:00002fc2       __exit                     00403fc2 f   msvcrt:MSVCRT.dll
 0001:00002fc8       __XcptFilter               00403fc8 f   msvcrt:MSVCRT.dll
 0001:00002fce       _exit                      00403fce f   msvcrt:MSVCRT.dll
 0001:00002fd4       ___p___initenv             00403fd4 f   msvcrt:MSVCRT.dll
 0001:00002fda       ___getmainargs             00403fda f   msvcrt:MSVCRT.dll
 0001:00002fe0       __initterm                 00403fe0 f   msvcrt:MSVCRT.dll
 0001:00002fe6       __setdefaultprecision      00403fe6 f   msvcrt:fp8.obj
 0001:00002ff8       ___setusermatherr          00403ff8 f   msvcrt:MSVCRT.dll
 0001:00002ffe       __matherr                  00403ffe f   msvcrt:merr.obj
 0001:00003001       __setargv                  00404001 f   msvcrt:dllargv.obj
 0001:00003002       ___p__commode              00404002 f   msvcrt:MSVCRT.dll
 0001:00003008       ___p__fmode                00404008 f   msvcrt:MSVCRT.dll
 0001:0000300e       __onexit                   0040400e f   msvcrt:atonexit.obj
 0001:0000303a       _atexit                    0040403a f   msvcrt:atonexit.obj
 0001:0000304c       ___set_app_type            0040404c f   msvcrt:MSVCRT.dll
 0001:00003052       __except_handler3          00404052 f   msvcrt:MSVCRT.dll
 0001:00003058       __controlfp                00404058 f   msvcrt:MSVCRT.dll
 0001:0000305e       ___dllonexit               0040405e f   msvcrt:MSVCRT.dll
 0001:00003064       _VerQueryValueA@16         00404064 f   Version:VERSION.dll
 0001:0000306a       _GetFileVersionInfoA@16    0040406a f   Version:VERSION.dll
 0001:00003070       _GetFileVersionInfoSizeA@8 00404070 f   Version:VERSION.dll
 0002:00000000       __imp__OutputDebugStringA@4 00405000     kernel32:KERNEL32.dll
 0002:00000004       __imp__GetTempPathA@8      00405004     kernel32:KERNEL32.dll
 0002:00000008       __imp__GetTickCount@0      00405008     kernel32:KERNEL32.dll
 0002:0000000c       __imp__LocalFree@4         0040500c     kernel32:KERNEL32.dll
 0002:00000010       __imp__FormatMessageA@28   00405010     kernel32:KERNEL32.dll
 0002:00000014       __imp__GetSystemDefaultLangID@0 00405014     kernel32:KERNEL32.dll
 0002:00000018       __imp__GetLastError@0      00405018     kernel32:KERNEL32.dll
 0002:0000001c       __imp__WideCharToMultiByte@32 0040501c     kernel32:KERNEL32.dll
 0002:00000020       __imp__GetProcAddress@8    00405020     kernel32:KERNEL32.dll
 0002:00000024       __imp__GetModuleHandleA@4  00405024     kernel32:KERNEL32.dll
 0002:00000028       __imp__FreeLibrary@4       00405028     kernel32:KERNEL32.dll
 0002:0000002c       __imp__LoadLibraryA@4      0040502c     kernel32:KERNEL32.dll
 0002:00000030       __imp__GetVersion@0        00405030     kernel32:KERNEL32.dll
 0002:00000034       __imp__GetVersionExA@4     00405034     kernel32:KERNEL32.dll
 0002:00000038       __imp__lstrcmpiA@8         00405038     kernel32:KERNEL32.dll
 0002:0000003c       __imp__GetVolumeInformationA@32 0040503c     kernel32:KERNEL32.dll
 0002:00000040       __imp__UnmapViewOfFile@4   00405040     kernel32:KERNEL32.dll
 0002:00000044       __imp__MapViewOfFile@20    00405044     kernel32:KERNEL32.dll
 0002:00000048       __imp__IsBadReadPtr@8      00405048     kernel32:KERNEL32.dll
 0002:0000004c       __imp__IsBadWritePtr@8     0040504c     kernel32:KERNEL32.dll
 0002:00000050       __imp__FileTimeToSystemTime@8 00405050     kernel32:KERNEL32.dll
 0002:00000054       __imp__GlobalMemoryStatusEx@4 00405054     kernel32:KERNEL32.dll
 0002:00000058       __imp__CloseHandle@4       00405058     kernel32:KERNEL32.dll
 0002:0000005c       __imp__GetCommandLineA@0   0040505c     kernel32:KERNEL32.dll
 0002:00000060       __imp__GetModuleFileNameA@12 00405060     kernel32:KERNEL32.dll
 0002:00000064       __imp__lstrcpynA@12        00405064     kernel32:KERNEL32.dll
 0002:00000068       __imp__VerLanguageNameA@12 00405068     kernel32:KERNEL32.dll
 0002:0000006c       \177KERNEL32_NULL_THUNK_DATA 0040506c     kernel32:KERNEL32.dll
 0002:00000070       __imp_??3@YAXPAX@Z         00405070     mfc42:MFC42.DLL
 0002:00000074       __imp_?AfxWinInit@@YGHPAUHINSTANCE__@@0PADH@Z 00405074     mfc42:MFC42.DLL
 0002:00000078       __imp_??0CDWordArray@@QAE@XZ 00405078     mfc42:MFC42.DLL
 0002:0000007c       __imp_?Delete@CString@@QAEHHH@Z 0040507c     mfc42:MFC42.DLL
 0002:00000080       __imp_??1CString@@QAE@XZ   00405080     mfc42:MFC42.DLL
 0002:00000084       __imp_?Right@CString@@QBE?AV1@H@Z 00405084     mfc42:MFC42.DLL
 0002:00000088       __imp_?ReleaseBuffer@CString@@QAEXH@Z 00405088     mfc42:MFC42.DLL
 0002:0000008c       __imp_?GetBuffer@CString@@QAEPADH@Z 0040508c     mfc42:MFC42.DLL
 0002:00000090       __imp_??0CString@@QAE@ABV0@@Z 00405090     mfc42:MFC42.DLL
 0002:00000094       __imp_?Format@CString@@QAAXPBDZZ 00405094     mfc42:MFC42.DLL
 0002:00000098       __imp_??0CString@@QAE@XZ   00405098     mfc42:MFC42.DLL
 0002:0000009c       __imp_??1CStdioFile@@UAE@XZ 0040509c     mfc42:MFC42.DLL
 0002:000000a0       __imp_?Close@CStdioFile@@UAEXXZ 004050a0     mfc42:MFC42.DLL
 0002:000000a4       __imp_?WriteString@CStdioFile@@UAEXPBD@Z 004050a4     mfc42:MFC42.DLL
 0002:000000a8       __imp_?Open@CStdioFile@@UAEHPBDIPAVCFileException@@@Z 004050a8     mfc42:MFC42.DLL
 0002:000000ac       __imp_??0CStdioFile@@QAE@XZ 004050ac     mfc42:MFC42.DLL
 0002:000000b0       __imp_?FormatV@CString@@QAEXPBDPAD@Z 004050b0     mfc42:MFC42.DLL
 0002:000000b4       __imp_?SetAtGrow@CDWordArray@@QAEXHK@Z 004050b4     mfc42:MFC42.DLL
 0002:000000b8       __imp_?Replace@CString@@QAEHPBD0@Z 004050b8     mfc42:MFC42.DLL
 0002:000000bc       __imp_??0CString@@QAE@PBD@Z 004050bc     mfc42:MFC42.DLL
 0002:000000c0       __imp_?SetSize@CDWordArray@@QAEXHH@Z 004050c0     mfc42:MFC42.DLL
 0002:000000c4       __imp_??1CDWordArray@@UAE@XZ 004050c4     mfc42:MFC42.DLL
 0002:000000c8       \177MFC42_NULL_THUNK_DATA  004050c8     mfc42:MFC42.DLL
 0002:000000cc       __imp___XcptFilter         004050cc     msvcrt:MSVCRT.dll
 0002:000000d0       __imp___onexit             004050d0     msvcrt:MSVCRT.dll
 0002:000000d4       __imp____dllonexit         004050d4     msvcrt:MSVCRT.dll
 0002:000000d8       __imp___mbscmp             004050d8     msvcrt:MSVCRT.dll
 0002:000000dc       __imp____CxxFrameHandler   004050dc     msvcrt:MSVCRT.dll
 0002:000000e0       __imp__wcslen              004050e0     msvcrt:MSVCRT.dll
 0002:000000e4       __imp__isalnum             004050e4     msvcrt:MSVCRT.dll
 0002:000000e8       __imp__printf              004050e8     msvcrt:MSVCRT.dll
 0002:000000ec       __imp__wcsncpy             004050ec     msvcrt:MSVCRT.dll
 0002:000000f0       __imp__free                004050f0     msvcrt:MSVCRT.dll
 0002:000000f4       __imp__strncpy             004050f4     msvcrt:MSVCRT.dll
 0002:000000f8       __imp__malloc              004050f8     msvcrt:MSVCRT.dll
 0002:000000fc       __imp__strncat             004050fc     msvcrt:MSVCRT.dll
 0002:00000100       __imp__strncmp             00405100     msvcrt:MSVCRT.dll
 0002:00000104       __imp__atoi                00405104     msvcrt:MSVCRT.dll
 0002:00000108       __imp__sscanf              00405108     msvcrt:MSVCRT.dll
 0002:0000010c       __imp___exit               0040510c     msvcrt:MSVCRT.dll
 0002:00000110       __imp___except_handler3    00405110     msvcrt:MSVCRT.dll
 0002:00000114       __imp__exit                00405114     msvcrt:MSVCRT.dll
 0002:00000118       __imp____p___initenv       00405118     msvcrt:MSVCRT.dll
 0002:0000011c       __imp____getmainargs       0040511c     msvcrt:MSVCRT.dll
 0002:00000120       __imp___initterm           00405120     msvcrt:MSVCRT.dll
 0002:00000124       __imp____setusermatherr    00405124     msvcrt:MSVCRT.dll
 0002:00000128       __imp___adjust_fdiv        00405128     msvcrt:MSVCRT.dll
 0002:0000012c       __imp____p__commode        0040512c     msvcrt:MSVCRT.dll
 0002:00000130       __imp____p__fmode          00405130     msvcrt:MSVCRT.dll
 0002:00000134       __imp____set_app_type      00405134     msvcrt:MSVCRT.dll
 0002:00000138       __imp___controlfp          00405138     msvcrt:MSVCRT.dll
 0002:0000013c       \177MSVCRT_NULL_THUNK_DATA 0040513c     msvcrt:MSVCRT.dll
 0002:00000140       __imp__ShellExecuteA@24    00405140     shell32:SHELL32.dll
 0002:00000144       \177SHELL32_NULL_THUNK_DATA 00405144     shell32:SHELL32.dll
 0002:00000148       __imp__wsprintfA           00405148     user32:USER32.dll
 0002:0000014c       \177USER32_NULL_THUNK_DATA 0040514c     user32:USER32.dll
 0002:00000150       __imp__GetFileVersionInfoA@16 00405150     Version:VERSION.dll
 0002:00000154       __imp__GetFileVersionInfoSizeA@8 00405154     Version:VERSION.dll
 0002:00000158       __imp__VerQueryValueA@16   00405158     Version:VERSION.dll
 0002:0000015c       \177VERSION_NULL_THUNK_DATA 0040515c     Version:VERSION.dll
 0002:0000017c       ??_7CFileVersionInfo@@6B@  0040517c     verinfo.obj
 0002:00000180       _IID_IDocHostUIHandlerDispatch 00405180     mfcs42:stdafx.obj
 0002:00000190       _IID_IInternalConnection   00405190     mfcs42:stdafx.obj
 0002:000001a0       _IID_IAxWinAmbientDispatch 004051a0     mfcs42:stdafx.obj
 0002:000001b0       _IID_IAxWinHostWindow      004051b0     mfcs42:stdafx.obj
 0002:000001c0       _IID_IRegistrar            004051c0     mfcs42:stdafx.obj
 0002:000001d0       _CLSID_Registrar           004051d0     mfcs42:stdafx.obj
 0002:000001e0       _LIBID_ATLLib              004051e0     mfcs42:stdafx.obj
 0002:00000438       __IMPORT_DESCRIPTOR_KERNEL32 00405438     kernel32:KERNEL32.dll
 0002:0000044c       __IMPORT_DESCRIPTOR_USER32 0040544c     user32:USER32.dll
 0002:00000460       __IMPORT_DESCRIPTOR_SHELL32 00405460     shell32:SHELL32.dll
 0002:00000474       __IMPORT_DESCRIPTOR_MFC42  00405474     mfc42:MFC42.DLL
 0002:00000488       __IMPORT_DESCRIPTOR_MSVCRT 00405488     msvcrt:MSVCRT.dll
 0002:0000049c       __IMPORT_DESCRIPTOR_VERSION 0040549c     Version:VERSION.dll
 0002:000004b0       __NULL_IMPORT_DESCRIPTOR   004054b0     kernel32:KERNEL32.dll
 0003:00000000       ___xc_a                    00406000     msvcrt:cinitexe.obj
 0003:00000018       ___xc_z                    00406018     msvcrt:cinitexe.obj
 0003:0000001c       ___xi_a                    0040601c     msvcrt:cinitexe.obj
 0003:00000020       ___xi_z                    00406020     msvcrt:cinitexe.obj
 0003:00000030       ??_C@_01PCFE@?2?$AA@       00406030     debugx.obj
 0003:00000034       ??_C@_0O@ONJB@?$CFs?2vin_?$CFd?4txt?$AA@ 00406034     debugx.obj
 0003:00000044       ??_C@_04KHOB@open?$AA@     00406044     debugx.obj
 0003:0000004c       ??_C@_07GOLH@notepad?$AA@  0040604c     debugx.obj
 0003:00000054       ??_C@_01BJG@?6?$AA@        00406054     debugx.obj
 0003:00000058       ??_C@_02MECO@?$CFd?$AA@    00406058     debugx.obj
 0003:0000005c       ??_C@_0P@NIOC@?$FL0x?$CF08X?$FN?5?$CFs?5?9?5?$AA@ 0040605c     debugx.obj
 0003:0000006c       ??_C@_02PIMC@?$AN?6?$AA@   0040606c     debugx.obj
 0003:00000070       ??_C@_02JBML@?$CFc?$AA@    00406070     debugx.obj
 0003:00000074       ??_C@_01PJCK@?4?$AA@       00406074     debugx.obj
 0003:00000078       ??_C@_05DLFD@?$CF02X?5?$AA@ 00406078     debugx.obj
 0003:00000080       ??_C@_01GJD@?9?$AA@        00406080     debugx.obj
 0003:00000084       ??_C@_06OFEH@?$CF08X?3?5?$AA@ 00406084     debugx.obj
 0003:0000008c       ??_C@_09MHEK@ntdll?4dll?$AA@ 0040608c     mem_nt.obj
 0003:00000098       ??_C@_0BF@LGHK@RtlInitUnicodeString?$AA@ 00406098     mem_nt.obj
 0003:000000b0       ??_C@_0BF@HAFJ@NtUnmapViewOfSection?$AA@ 004060b0     mem_nt.obj
 0003:000000c8       ??_C@_0O@OBIL@NtOpenSection?$AA@ 004060c8     mem_nt.obj
 0003:000000d8       ??_C@_0BD@LLBJ@NtMapViewOfSection?$AA@ 004060d8     mem_nt.obj
 0003:000000ec       ??_C@_0BG@NCLP@RtlNtStatusToDosError?$AA@ 004060ec     mem_nt.obj
 0003:00000104       ??_C@_0BF@GEIA@MmGetPhysicalAddress?$AA@ 00406104     mem_nt.obj
 0003:0000011c       ??_C@_0N@FFHM@ntoskrnl?4exe?$AA@ 0040611c     mem_nt.obj
 0003:0000012c       ??_C@_04GDDA@NTFS?$AA@     0040612c     mem_os.obj
 0003:00000134       ??_C@_07OEOL@?$CFs?3?5?$CFs?6?$AA@ 00406134     mem_phys.obj
 0003:0000013c       ??_C@_0CG@MAAJ@Could?5not?5open?5?2device?2physicalm@ 0040613c     mem_phys.obj
 0003:00000164       ??_C@_1CO@LFHG@?$AA?2?$AAd?$AAe?$AAv?$AAi?$AAc?$AAe?$AA?2?$AAp?$AAh?$AAy?$AAs?$AAi?$AAc?$AAa?$AAl?$AAm?$AAe?$AAm?$AAo@ 00406164     mem_phys.obj
 0003:00000194       ??_C@_0BF@BKLB@Unable?5to?5unmap?5view?$AA@ 00406194     mem_phys.obj
 0003:000001ac       ??_C@_0BG@EICC@Starting?5Hivelist?4?4?4?6?$AA@ 004061ac     mem_reg.obj
 0003:000001c4       ??_C@_0EC@ILL@Last?5modification?5time?3?5?$CF02d?1?$CF02@ 004061c4     mem_reg.obj
 0003:00000208       ??_C@_01FCOA@?5?$AA@       00406208     mem_reg.obj
 0003:0000020c       ??_C@_0GL@NNMJ@?$CF?42s?3?5type?50x?$CFx?5parent?50x?$CFx?0?5?$CFd?5@ 0040620c     mem_reg.obj
 0003:00000278       ??_C@_0BB@LHPH@?$CFsCell?3?5li?5?$CI?$CFd?$CJ?6?$AA@ 00406278     mem_reg.obj
 0003:0000028c       ??_C@_0BB@MEIN@?$CFsCell?3?5ri?5?$CI?$CFd?$CJ?6?$AA@ 0040628c     mem_reg.obj
 0003:000002a0       ??_C@_0N@MFBJ@?$CFsCell?3?5sk?0?5?$AA@ 004062a0     mem_reg.obj
 0003:000002b0       ??_C@_0N@HFAD@?$CFsCell?3?5vk?0?5?$AA@ 004062b0     mem_reg.obj
 0003:000002c0       ??_C@_0BP@JEKE@?$CFs?5RootCell?30x?$CFx?0?5Hive?30x?$CF08X?6?$AA@ 004062c0     mem_reg.obj
 0003:000002e0       ??_C@_0N@EABG@?$CFsCell?3?5lk?0?5?$AA@ 004062e0     mem_reg.obj
 0003:000002f0       ??_C@_0BB@JJGC@?$CFsCell?3?5lh?5?$CI?$CFd?$CJ?6?$AA@ 004062f0     mem_reg.obj
 0003:00000304       ??_C@_0BB@KLC@?$CFsCell?3?5lf?5?$CI?$CFd?$CJ?6?$AA@ 00406304     mem_reg.obj
 0003:00000318       ??_C@_0BF@EAJI@?$CFsCell?3?5nk?0?5?$CFs?5?$CI?$CFd?$CJ?6?$AA@ 00406318     mem_reg.obj
 0003:00000330       ??_C@_01FCCL@?$CF?$AA@     00406330     mem_reg.obj
 0003:00000334       ??_C@_02MLHJ@?$CF?$CF?$AA@ 00406334     mem_reg.obj
 0003:00000338       ??_C@_0BE@MEPO@?$CFsCell?3?5Deleted?4?$CFs?6?$AA@ 00406338     mem_reg.obj
 0003:0000034c       ??_C@_09LEAC@?5?5?5?9?9?9?9?9?6?$AA@ 0040634c     mem_reg.obj
 0003:00000358       ??_C@_0BN@LNKH@?5?5?5Finded?5Base?5block?50x?$CF08X?6?$AA@ 00406358     mem_reg.obj
 0003:00000378       ??_C@_0CL@FBEC@?5?5?5?$DM?$DM?$DMErr?$DO?$DO?$DO?5Invalid?5BaseBlock?5S@ 00406378     mem_reg.obj
 0003:000003a4       ??_C@_04JKI@Flat?$AA@      004063a4     mem_reg.obj
 0003:000003ac       ??_C@_0O@PGPF@?70x?$CF08X?5?5?$CFls?6?$AA@ 004063ac     mem_reg.obj
 0003:000003bc       ??_C@_0BK@KHML@?5?5?$CF02d?$CJ?5Hive?5Version?3?5?$CFld?$AA@ 004063bc     mem_reg.obj
 0003:000003d8       ??_C@_08OLGF@?5?5?$CF02d?$CJ?6?$AA@ 004063d8     mem_reg.obj
 0003:000003e4       ??_C@_0BG@FJFF@Starting?5MakeTree?4?4?4?6?$AA@ 004063e4     mem_reg.obj
 0003:000003fc       ??_C@_0CK@IPLC@?5?5?$DM?$DM?$DMErr?$DO?$DO?$DO?5Fail?5to?5read?5unicode@ 004063fc     mem_reg.obj
 0003:00000428       ??_C@_0BI@GGKF@?5?5?$CF02d?$CJ?50x?$CF08I64X?5?5?$CFls?6?$AA@ 00406428     mem_reg.obj
 0003:00000440       ??_C@_1BE@HAK@?$AA?$DM?$AAN?$AAo?$AA?5?$AAN?$AAa?$AAm?$AAe?$AA?$DO?$AA?$AA@ 00406440     mem_reg.obj
 0003:00000454       ??_C@_0DB@HJKM@Found?5?$CFd?5PoolTag?$CIs?$CJ?5of?5Windows?5R@ 00406454     mem_reg.obj
 0003:00000488       ??_C@_04LDIA@Idle?$AA@     00406488     mem_x86.obj
 0003:00000490       ?g_rgOptions@@3PAUSOption@?$CSimpleOptTempl@D@@A 00406490     regwipe.obj
 0003:000004d0       ??_C@_04MHDN@help?$AA@     004064d0     regwipe.obj
 0003:000004d8       ??_C@_07KNLF@verbose?$AA@  004064d8     regwipe.obj
 0003:000004e0       ??_C@_08GDIA@loglevel?$AA@ 004064e0     regwipe.obj
 0003:000004ec       ??_C@_0M@IBML@?$CFd?4?$CFd?4?$CFd?4?$CFd?$AA@ 004064ec     regwipe.obj
 0003:000004f8       ??_C@_0CCL@FKLJ@Usage?3?5CowboyC?5?$FLOPTION?$FN?4?4?4?5?$FLPATH@ 004064f8     regwipe.obj
 0003:00000724       ??_C@_0DA@EFDM@RegWipe?5v?$CFs?0?5Windows?5physical?5me@ 00406724     regwipe.obj
 0003:00000754       ??_C@_0CG@LDNA@?5?9?$DO?5ERROR?3?5Not?5Supported?5OS?4Sorr@ 00406754     regwipe.obj
 0003:0000077c       ??_C@_0CC@CLAP@Memory?5Total?5Size?3?50x?$CFI64X?5Bytes@ 0040677c     regwipe.obj
 0003:000007a0       ??_C@_0CM@MEGF@?5?9?$DO?5ERROR?3?5GlobalMemoryStatusEx?5@ 004067a0     regwipe.obj
 0003:000007cc       ??_C@_0DC@KLLJ@?5?9?$DO?5ERROR?3?5Unable?5to?5locate?5NTDL@ 004067cc     regwipe.obj
 0003:00000800       ??_C@_0BH@FAGI@Success?5init?5process?4?6?$AA@ 00406800     regwipe.obj
 0003:00000818       ??_C@_0BP@DCJG@Success?5Open?5physical?5memory?4?6?$AA@ 00406818     regwipe.obj
 0003:00000838       ??_C@_0DA@MNAN@?$CFs?3?5?8?$CFs?8?5?$CIuse?5?9?9help?5to?5get?5comm@ 00406838     regwipe.obj
 0003:00000868       ??_C@_0BN@MBCL@Required?5argument?5is?5missing?$AA@ 00406868     regwipe.obj
 0003:00000888       ??_C@_0BI@OEMJ@Invalid?5argument?5format?$AA@ 00406888     regwipe.obj
 0003:000008a0       ??_C@_0CA@POEA@Option?5does?5not?5accept?5argument?$AA@ 004068a0     regwipe.obj
 0003:000008c0       ??_C@_0CA@BHMM@Option?5matched?5multiple?5strings?$AA@ 004068c0     regwipe.obj
 0003:000008e0       ??_C@_0BE@BHNK@Unrecognized?5option?$AA@ 004068e0     regwipe.obj
 0003:000008f4       ??_C@_0O@NOFB@Unknown?5error?$AA@ 004068f4     regwipe.obj
 0003:00000904       ??_C@_02JDLK@?$CFx?$AA@    00406904     regwipe.obj
 0003:00000908       ?s_ppszStr@CFileVersionInfo@@1PAPBDA 00406908     verinfo.obj
 0003:0000093c       ??_C@_0BA@KHPE@OLESelfRegister?$AA@ 0040693c     verinfo.obj
 0003:0000094c       ??_C@_0N@IOKF@SpecialBuild?$AA@ 0040694c     verinfo.obj
 0003:0000095c       ??_C@_0P@JKBO@ProductVersion?$AA@ 0040695c     verinfo.obj
 0003:0000096c       ??_C@_0M@OKED@ProductName?$AA@ 0040696c     verinfo.obj
 0003:00000978       ??_C@_0N@EHDI@PrivateBuild?$AA@ 00406978     verinfo.obj
 0003:00000988       ??_C@_0BB@JMFD@OriginalFilename?$AA@ 00406988     verinfo.obj
 0003:0000099c       ??_C@_0BA@NHED@LegalTrademarks?$AA@ 0040699c     verinfo.obj
 0003:000009ac       ??_C@_0P@NIMM@LegalCopyright?$AA@ 004069ac     verinfo.obj
 0003:000009bc       ??_C@_0N@CCA@InternalName?$AA@ 004069bc     verinfo.obj
 0003:000009cc       ??_C@_0M@EOAE@FileVersion?$AA@ 004069cc     verinfo.obj
 0003:000009d8       ??_C@_0BA@EJP@FileDescription?$AA@ 004069d8     verinfo.obj
 0003:000009e8       ??_C@_0M@HFKG@CompanyName?$AA@ 004069e8     verinfo.obj
 0003:000009f4       ??_C@_08JMHK@Comments?$AA@ 004069f4     verinfo.obj
 0003:00000a00       ??_C@_0BJ@KCFH@?2VarFileInfo?2Translation?$AA@ 00406a00     verinfo.obj
 0003:00000a1c       ??_C@_0BM@DEAI@?2StringFileInfo?2?$CF04X?$CF04X?2?$CFs?$AA@ 00406a1c     verinfo.obj
 0003:00000a38       ??_C@_07PCHH@Unknown?$AA@  00406a38     verinfo.obj
 0003:00000a40       ??_C@_06NOBP@Arabic?$AA@   00406a40     verinfo.obj
 0003:00000a48       ??_C@_06CGFP@Hebrew?$AA@   00406a48     verinfo.obj
 0003:00000a50       ??_C@_07MPOO@Turkish?$AA@  00406a50     verinfo.obj
 0003:00000a58       ??_C@_05DKAJ@Greek?$AA@    00406a58     verinfo.obj
 0003:00000a60       ??_C@_0N@GEIL@Multilingual?$AA@ 00406a60     verinfo.obj
 0003:00000a70       ??_C@_08JMMJ@Cyrillic?$AA@ 00406a70     verinfo.obj
 0003:00000a7c       ??_C@_07NCOA@Unicode?$AA@  00406a7c     verinfo.obj
 0003:00000a84       ??_C@_0BL@MOJH@Latin?92?5?$CIEastern?5European?$CJ?$AA@ 00406a84     verinfo.obj
 0003:00000aa0       ??_C@_0O@GGA@Taiwan?5?$CIBig5?$CJ?$AA@ 00406aa0     verinfo.obj
 0003:00000ab0       ??_C@_0M@HEFK@7?9bit?5ASCII?$AA@ 00406ab0     verinfo.obj
 0003:00000abc       ??_C@_0BL@OPDI@Japan?5?$CIShift?5?$JG?5JIS?5X?90208?$CJ?$AA@ 00406abc     verinfo.obj
 0003:00000ad8       ??_C@_0BJ@BCOG@Korea?5?$CIShift?5?$JG?5KSC?55601?$CJ?$AA@ 00406ad8     verinfo.obj
 0003:00000af8       ?GUID_ATLVer30@ATL@@3U_GUID@@A 00406af8     mfcs42:stdafx.obj
 0003:00000b10       ___defaultmatherr          00406b10     msvcrt:merr.obj
 0003:00000b18       ?g_pODSProc@@3P6AXPBD@ZA   00406b18     debugx.obj
 0003:00000b1c       ?g_fnMmGetPhysicalAddress@@3P6G?AT_LARGE_INTEGER@@PAX@ZA 00406b1c     mem_nt.obj
 0003:00000b20       ?g_fnNtUnmapViewOfSection@@3P6GJPAX0@ZA 00406b20     mem_nt.obj
 0003:00000b24       ?g_fnRtlNtStatusToDosError@@3P6GKJ@ZA 00406b24     mem_nt.obj
 0003:00000b28       ?g_fnNtMapViewOfSection@@3P6GJPAX0PAPAXKKPAT_LARGE_INTEGER@@PAKW4_SECTION_INHERIT@@KK@ZA 00406b28     mem_nt.obj
 0003:00000b2c       ?g_fnRtlInitUnicodeString@@3P6GXPAU_UNICODE_STRING@@PBG@ZA 00406b2c     mem_nt.obj
 0003:00000b30       ?g_fnNtOpenSection@@3P6GJPAPAXKPAU_OBJECT_ATTRIBUTES@@@ZA 00406b30     mem_nt.obj
 0003:00000b38       ?g_dwDTB@@3KA              00406b38     regwipe.obj
 0003:00000b40       ?g_ullTotalPhys@@3_KA      00406b40     regwipe.obj
 0003:00000b48       ?g_bVerbose@@3HA           00406b48     regwipe.obj
 0003:00000b4c       ?g_nWinXPSP@@3GA           00406b4c     regwipe.obj
 0003:00000b4e       ?g_nLogLevel@@3FA          00406b4e     regwipe.obj
 0003:00000b50       __afxForceEXCLUDE          00406b50     mfcs42:nolib.obj
 0003:00000b54       ?ATL_CREATE_OBJECT@CComApartment@ATL@@2IA 00406b54     mfcs42:stdafx.obj
 0003:00000b58       ?m_libid@CComModule@ATL@@2U_GUID@@A 00406b58     mfcs42:stdafx.obj
 0003:00000b68       ?_pModule@ATL@@3PAVCComModule@1@A 00406b68     mfcs42:stdafx.obj
 0003:00000b6c       __afxForceSTDAFX           00406b6c     mfcs42:stdafx.obj
 0003:00000b70       __dowildcard               00406b70     msvcrt:wildcard.obj
 0003:00000b74       __newmode                  00406b74     msvcrt:_newmode.obj
 0003:00000b78       __commode                  00406b78     msvcrt:xncommod.obj
 0003:00000b7c       __fmode                    00406b7c     msvcrt:xtxtmode.obj
 0003:00000b80       ___onexitend               00406b80     <common>
 0003:00000b84       ___onexitbegin             00406b84     <common>
 0003:00000b88       __adjust_fdiv              00406b88     <common>

 entry point at        0001:00002eb2

 Static symbols

 0001:000007a0       _$E201                     004017a0 f   mem_nt.obj
 0001:000007b0       _$E200                     004017b0 f   mem_nt.obj
 0001:000007d0       _$E204                     004017d0 f   mem_nt.obj
 0001:000007e0       _$E203                     004017e0 f   mem_nt.obj
 0001:00000800       _$E207                     00401800 f   mem_nt.obj
 0001:00000810       _$E206                     00401810 f   mem_nt.obj
 0001:00000830       _$E210                     00401830 f   mem_nt.obj
 0001:00000840       _$E209                     00401840 f   mem_nt.obj
 0001:00000860       _$E213                     00401860 f   mem_nt.obj
 0001:00000870       _$E212                     00401870 f   mem_nt.obj
